S023000062696E2F6F70656E626C745F6F6C696D6578696E6F5F73746D33322E737265635A
S3150800000000500020BD010008030200080502000890
S3150800001007020008090200080B0200080000000099
S315080000200000000000000000000000000D020008AB
S315080000300F02000800000000110200081302000861
S3150800004017020008190200081B0200081D02000812
S315080000501F020008210200082302000825020008E2
S3150800006027020008290200082B0200082D020008B2
S315080000702F02000831020008330200083502000882
S3150800008037020008390200083B0200083D02000852
S315080000903F02000841020008430200084502000822
S315080000A047020008490200084B0200084D020008F2
S315080000B04F020008510200085302000855020008C2
S315080000C057020008590200085B0200085D02000892
S315080000D05F02000861020008630200086502000862
S315080000E067020008690200086B02000810B5054C93
S315080000F0237833B9044B13B10448AFF300800123C6
S31508000100237010BDC802002000000000885C0008AB
S31508000110084B10B51BB108490848AFF300800848DA
S31508000120036803B910BD074B002BFBD0BDE8104090
S31508000130184700BF00000000CC020020885C0008B9
S31508000140C802002000000000154B002B08BF134B07
S315080001509D46A3F5803A00218B460F461348144A5C
S31508000160121A05F001F90F4B002B00D098470E4BD9
S31508000170002B00D098470020002104000D000D48F0
S31508000180002802D00C48AFF3008005F09FF8200045
S31508000190290000F047F905F085F800BF00000800BF
S315080001A0005000200000000000000000C8020020E7
S315080001B0B2130020000000000000000006498D462A
S315080001C00649074A074B9A42BEBF51F8040B42F844
S315080001D0040BF8E70448004700500020945C000828
S315080001E000000020C8020020490100081F49204AD3
S315080001F0002301E041F8043B9142FBD300F012F9D9
S31508000200FEE7FEE7FEE7FEE7FEE7FEE7FEE7FEE7B8
S31508000210FEE7FEE7FEE7FEE7FEE7FEE7FEE7FEE7A8
S31508000220FEE7FEE7FEE7FEE7FEE7FEE7FEE7FEE798
S31508000230FEE7FEE7FEE7FEE7FEE7FEE7FEE7FEE788
S31508000240FEE7FEE7FEE7FEE7FEE7FEE7FEE7FEE778
S31508000250FEE7FEE7FEE7FEE7FEE7FEE7FEE7FEE768
S31508000260FEE7FEE7FEE7FEE7FEE7FEE7C802002038
S31508000270B213002002F0B4BD02F0F8BD034B1B68B0
S31508000280052B00D0704702F0ABBD00BF2405002047
S31508000290034B9B7A13B1034B05221A60704700BFC4
S315080002A08413002024050020014B04221A6070479D
S315080002B024050020704700BF062801D00220704799
S315080002C00B4B1B681A7802F07F02012AF6D110B58B
S315080002D05C7954B99A78212A07D1064A5C829A61D0
S315080002E0204600F097F8204610BD022010BD00BF3A
S315080002F0A4130020150400080220704709B1022043
S315080003007047002814BF02200020704710B502F07D
S31508000310D3FD054B00241B689C7201F03DFE00F0DE
S3150800032085FF024B1C6010BDA41300202405002085
S3150800033010B5264B264A1B68D27900245A729C723D
S31508000340DC72204600F096FF20464FF4007100F05C
S3150800035099FF2046102100F0A3FF2046402101F016
S3150800036083F88021204601F06DF8204601F004F854
S31508000370184B204693F82C1001F032F8204600F06E
S31508000380D7FF2146012000F07DFF4FF48071012040
S3150800039001F058F8C021012001F066F8402101203B
S315080003A001F010F84021012001F01AF84FF44051ED
S315080003B0012000F08FFF2021012000F071FF204668
S315080003C001F000FD044B01221A6010BDA4130020A1
S315080003D0EC5300082400002024050020014901F000
S315080003E041BA00BF80000020014901F03BBA00BFB6
S315080003F01C000020054B1B68DB78052B04D8044934
S3150800040001EBC30101F02EBA00207047A4130020A7
S3150800041088000020014901F025BA00BF78000020B5
S31508000420704700BF00B5534B002285B00192029277
S315080004301968514A41F0010119605D684FF41F01BE
S315080004402A405A601A6840F2DC5422F0847222F478
S3150800045080321A601A68184622F480221A605A688E
S3150800046022F4FE025A6099601A6842F480321A60D1
S3150800047002E0019BA34209D0036803F40033029308
S31508000480019B01330193029B002BF2D0394B1B6869
S3150800049099036AD5394A374B1068194640F0100057
S315080004A01060106820F003001060106840F0020029
S315080004B010605A685A605A6842F400525A605A687C
S315080004C042F480625A605A6822F47C125A605A686A
S315080004D042F4E8125A601A6842F080721A600A6892
S315080004E0244B9201FBD519465A6822F003025A603A
S315080004F05A6842F002025A604A681E4B02F00C0221
S31508000500082AF9D101210D465A6804AC22F4800262
S315080005105A60DA69042042F40002DA6100F072FDDA
S3150800052024F8045D48232146032615488DF80F3024
S315080005308DF80E6000F0CAFD2946042000F062FD21
S315080005402025102321460E488DF80F308DF80E60B1
S31508000550ADF80C5000F0BAFD2946094800F024FE13
S3150800056001F040FF01F050FFFCE76F21054802F05B
S3150800057011FB8FE7001002400000FFF80020024040
S31508000580000801405454000830B5154C83B0237850
S31508000590054643B1012D4FF4805112481CD000F096
S315080005A001FE03B030BD0121102000F02BFD02A989
S315080005B04FF4805321F8043D0322142309488DF88B
S315080005C007308DF8062000F081FD0123012D2370E8
S315080005D04FF480510348E2D100F0E6FD03B030BD88
S315080005E0100500200010014008B50121034800F05D
S315080005F0D3FD10B100F0A2F8012008BD00080140A3
S31508000600642000F06FB800BF00F072B800B5C7B03C
S31508000610002168464FF48C7204F0A6FE6946094824
S3150800062004F0F0FC50B9009828B19DF8080080F055
S315080006301000C0F3001047B05DF804FB002047B077
S315080006405DF804FB5C540008004870475C540008D9
S3150800065010B5074C002320460A22064984F828329A
S3150800066004F052F910B9012384F8283210BD00BFEE
S31508000670E40200207C54000808B5084890F828329F
S31508000680012B04D0BDE80840054804F0EBBC04F093
S31508000690F5FBBDE80840024804F0E4BCE40200208B
S315080006A05C540008034890F82832012B00D07047A4
S315080006B004F0E4BBE402002010B5094C94F8283293
S315080006C0012B00D010BD214604F050FD0028F9DAB0
S315080006D0002384F828322046BDE8104004F0CEBB3B
S315080006E0E4020020014B1880704700BF1205002065
S315080006F010B502F099FE0D4C236898420ED30C4BA8
S315080007001A7862B1002220210A481A7000F04CFDBE
S3150800071002F08AFE084B1B881844206010BD01228F
S31508000720202104481A7000F03DFDF1E71405002069
S31508000730110500200008014012050020202101486B
S3150800074000F032BD0008014070B51749174C0B6818
S31508000750174D9BB2238022882B881A40920517D4FE
S31508000760228802F4004213420ED1228802F48062E3
S31508000770134200D170BD4FF6FF310B4A0D4B116085
S315080007805B68BDE87040184701F03EFB2B88ECE734
S315080007904FF6FF53084A0B6013780133DBB2137028
S315080007A0FFF76CFD2B88DBE7445C004074130020E0
S315080007B0A81300202400002018050020014608B5CB
S315080007C0064800F069FC0121044800F079FC00287D
S315080007D0F9D0024800F062FCC0B208BD00380040FB
S315080007E010B502F021FE00F5FA7403E002F01CFED3
S315080007F0844206D9FF20FFF7E1FFFF28F6D1012042
S3150800080010BD002010BD00BF10B504210A4800F035
S31508000810CBFCFF20FFF7D2FFFFF7E2FF10B1012460
S31508000820204610BD04460421034800F0BBFCFF2007
S31508000830FFF7C4FF204610BD0014014038B50D4629
S31508000840010604460BD40421224800F0ABFCFF2025
S31508000850FFF7B4FFFFF7D8FF58B9FF2038BD0021CE
S315080008603720FFF7EBFF012800D938BD04F07F04D5
S31508000870E9E744F04000FFF7A1FF280EFFF79EFFC7
S31508000880C5F30740FFF79AFFC5F30720FFF796FF62
S31508000890E8B2FFF793FF2CB1082C12D18720FFF797
S315080008A08DFF02E09520FFF789FF0A24FF20FFF756
S315080008B085FF020604F1FF33D7D513F0FF04F5D1FF
S315080008C038BD0120FFF77AFF0C2CEED1FF20FFF789
S315080008D075FFEAE70014014070B504460D4602F0BC
S315080008E0A3FD00F1640603E002F09EFD86421DD9D1
S315080008F0FF20FFF763FFFF28F6D0FE2816D1023443
S31508000900FF20FFF75BFF04F8020CFF20FFF756FFF6
S31508000910023D04F8010C04F10204F1D1FF20FFF7AF
S315080009204DFFFF20FFF74AFF012070BD002070BD74
S3150800093038B505460C46FFF753FF00B938BD2046C3
S31508000940FFF73CFFFD2C1ED0AC1C05F2022514F85F
S31508000950020CFFF733FF023414F8030CFFF72EFFDF
S31508000960AC42F4D1FF20FFF729FFFF20FFF726FF4F
S31508000970FF20FFF723FF00F01F00A0F10500B0FAE3
S3150800098080F0400938BD0120D8E700BF002840F0B4
S31508000990C2802DE9F043AC4D89B02B7803F00203F1
S315080009A003F0FF0423B12878C0B209B0BDE8F0838C
S315080009B00121202000F026FB01210820042700F051
S315080009C021FB01214FF4804000F02AFB03260DEBA2
S315080009D007014FF010099D48ADF804708DF807908F
S315080009E08DF8066000F072FB3946984800F0DAFB8D
S315080009F04FF4204218230DEB07019548ADF8042063
S31508000A008DF807308DF8066000F060FB4FF48042E1
S31508000A1048230DEB07018E48ADF804208DF8073002
S31508000A200DF10C0800F052FB4FF482724FF400737C
S31508000A304146ADF80E20ADF8163038220723854812
S31508000A40ADF81820ADF81C30ADF80C40ADF81040E4
S31508000A50ADF81240ADF81440ADF81A4000F0EEFAC1
S31508000A6021467C4800F01EFB01217A4800F006FB6F
S31508000A703946764800F096FB4FF4004402A97448BC
S31508000A80ADF808408DF80A608DF80B9000F01EFB53
S31508000A9021466F4800F086FB0A2402216D4800F0C3
S31508000AA00FFB0028F9D0FF216A4800F0F5FA01216A
S31508000AB0684800F005FB0028F9D0013CEDD14FF459
S31508000AC000400322182302A9ADF8080060488DF8F3
S31508000AD00A208DF80B3000F0F9FA04215B4800F083
S31508000AE063FB21462046FFF7A9FE0128064614D0D7
S31508000AF0594B0022042155481A6000F053FBFF2089
S31508000B00FFF75CFE2B7843F001032B702878C0B200
S31508000B1009B0BDE8F0830120704702F085FC4FF468
S31508000B20D57100F57A770820FFF788FE012835D1B8
S31508000B3002AC2646FF20FFF741FE06F8010BB0453A
S31508000B40F8D19DF80A30012BD2D19DF80B30AA2B8B
S31508000B50CED102E0FFF772FE38B102F065FC87429B
S31508000B604FF080414FF0A900F4D802F05DFC8742AF
S31508000B70BED900213A20FFF761FE0028B8D1FF2030
S31508000B80FFF71CFE04F8010BA045F8D19DF80830C4
S31508000B9013F0400F14BF0C2604261EE02146A92098
S31508000BA0FFF74CFE01289ABF0226A924344603E023
S31508000BB02046FFF743FE28B102F036FC87424FF085
S31508000BC00001F5D802F030FC874291D94FF4007144
S31508000BD01020FFF733FE00288AD11F4B04211B483B
S31508000BE01E6000F0DFFAFF20FFF7E8FD00210C4643
S31508000BF02B78184803F0FE032B704FF4827700F029
S31508000C003DFA4FF400760822072341461148ADF80D
S31508000C101820ADF81C30ADF80C40ADF81040ADF812
S31508000C201240ADF81440ADF81A40ADF80E70ADF8A4
S31508000C30166000F003FA2146064800F033FA01214F
S31508000C40044800F01BFAAEE6EC0000200014014050
S31508000C50000C0140003800401C05002018B9034B61
S31508000C601878C0B270470120704700BFEC0000201A
S31508000C7010B582B018B10424204602B010BD002B6E
S31508000C80F9D00C4620490978C80701D50324F3E7AB
S31508000C901E4901930968090758BF5202012B1146DC
S31508000CA020D01220FFF7CAFD019B58B10124042168
S31508000CB0174800F077FAFF20FFF780FDDCE7019B75
S31508000CC0013B16D020464FF400710193FFF704FE4E
S31508000CD004F500740028F2D1012400210C20FFF746
S31508000CE0ADFDE4E71120FFF7A9FD019B18B11C46ED
S31508000CF0DDE71C46F1E720464FF40071FFF7ECFDEF
S31508000D00B0FA80F46409D2E7EC0000201C05002044
S31508000D100014014010B582B018B10424204602B070
S31508000D2010BD002BF9D00C462A490878C00701D512
S31508000D300324F3E70978490701D50224EEE7264993
S31508000D400968080758BF5202012B35D011F0060F63
S31508000D5029D1114619200093FFF770FD009B50B169
S31508000D60012404211D4800F01DFAFF20FFF726FD87
S31508000D70D4E7013B09D02046FC210093FFF7D8FDB4
S31508000D8004F50074009B0028F3D10093FFF728FDB3
S31508000D90009B0028E4D01C1C4FF0FD0018BF01245E
S31508000DA0FFF70CFDDDE71946972001920093FFF740
S31508000DB045FD019A009BCCE711461820FFF73EFD3A
S31508000DC00028CDD12046FE21FFF7B2FDB0FA80F407
S31508000DD06409C6E7EC0000201C0500200014014049
S31508000DE008B104207047834B1B78D80701D5032028
S31508000DF0704770B5154684B00E2900F2A380DFE867
S31508000E0001F05F65A129A1A1A1A1A1A15A4C991838
S31508000E100800794B1B685B0700F1B980012404219F
S31508000E20764800F0BFF9FF20FFF7C8FC204604B05B
S31508000E3070BD00213A20FFF701FD0028EED16C1E97
S31508000E400335FF20FFF7BAFC04F8010FAC42F8D1CE
S31508000E500024E4E7684E336813F0040174D00021D7
S31508000E608D20FFF7EBFC0028D8D1FF20FFF7A6FC62
S31508000E7010216846FFF730FD0028CFD03024FF2028
S31508000E80FFF79CFC601E10F0FF04F8D19DF80A20BD
S31508000E901023120993402B60C1E700210920FFF7B0
S31508000EA0CDFC0028BAD128461021FFF715FDB0FA67
S31508000EB080F46409B3E7504B00241B681370AEE74F
S31508000EC0FFF7A2FCB0FA80F46409A8E7002109201C
S31508000ED0FFF7B4FC04460028A0D110216846FFF7A6
S31508000EE0FBFC00289AD09DF800309B09012B60D0A6
S31508000EF09DF805309DF80A609DF8092003F00F015A
S31508000F009DF807009DF8063001EBD61152009DF8B2
S31508000F100860023102F0060280009B020A4403F4CC
S31508000F20406300EB9611D2B20B44093A0133934061
S31508000F302B6074E700210A20FFF780FC00287FF465
S31508000F406DAFB0E704246AE70920FFF777FC04468B
S31508000F5000287FF463AF10216846FFF7BDFC002820
S31508000F603FF45CAF336813F0020332D09DF80A30C1
S31508000F709DF80B105B009DF80D2003F07E0303EB34
S31508000F80D11392090133013A93402B6047E70021B8
S31508000F908D20FFF753FC00287FF440AFFF20FFF7B2
S31508000FA00DFC28464021FFF797FCB0FA80F4640947
S31508000FB035E79DF807309DF808101B049DF80920B1
S31508000FC003F47C13013302EB012213449B022B60CA
S31508000FD025E79DF80B409DF80A20E00000F0180070
S31508000FE0C2F3840100EB54104A1C00FB02221C4683
S31508000FF02A6014E7EC0000201C05002000140140BC
S31508001000FEE700BF29B9054A936923EA0000906103
S315080010107047024B9A691043986170470010024066
S3150800102029B9054AD36923EA0000D0617047024B03
S31508001030DA691043D8617047001002404A8830B414
S315080010400C888B882243CC881A430B8922434C8907
S315080010508D891A4322430388CC892A43224303F401
S31508001060415313439BB20380838B30BC23F4006344
S315080010701B041B0C83830B8A03827047038829B9D8
S3150800108023F040031B041B0C038070479BB243F0FC
S3150800109040030380704700BF81817047808980B212
S315080010A0704700BF038829B923F400531B041B0C9F
S315080010B0038070479BB243F400530380704700BF18
S315080010C00389194214BF012000207047CB782DE907
S315080010D0F04103F00F06DB0648BF8B780C8848BF43
S315080010E01E4314F0FF0F26D00568002301274FF092
S315080010F00F0803E00133082B1BD00C8807FA03F20C
S3150800110032EA0404F6D19C0091F803E008FA04FCDC
S3150800111025EA0C0506FA04F4BEF1280F45EA04058B
S3150800112038D0BEF1480F03F1010308BF0261082B4E
S31508001130E3D105600C88FF2C2AD9456800230127CE
S315080011404FF00F0C03E00133082B20D00C8803F175
S31508001150080207FA02F232EA0404F4D191F803E02D
S315080011609C00BEF1280F04BF426191F803E00CFA17
S3150800117004F8BEF1480F03F1010325EA080506FA4B
S3150800118004F408BF0261082B45EA0405DED1456070
S31508001190BDE8F0814261ADE78368194214BF0120BA
S315080011A00020704701617047416170470132521053
S315080011B00ED010B401F1005101F540514900002349
S315080011C030F8024B21F8234001339A42F8D110BC7B
S315080011D0704700BF01F10051013201F5405152102C
S315080011E04FEA410105D051F8043B013A20F8023B89
S315080011F0F9D1704770B4074A07490848084E094CA0
S31508001200094B022515720860236032601B6870BCA2
S31508001210184700BF84130020A013002054000020A4
S31508001220A41300207C1300202400002010B40549D4
S31508001230054C064A00204FF4064320600B801360D5
S3150800124010BC7047A8130020445C0040405C004076
S3150800125070B500F07F0528460E4600F037F90446BB
S31508001260284600F021F9224601463046FFF7B2FF2C
S31508001270204670BD4FF6F873014A03401360704765
S31508001280505C0040800000F1804000F5B8400368DB
S3150800129023F4EC4323F07003194389B201607047C5
S315080012A0800000F1804000F5B8400368CA0623F4C0
S315080012B0E04323F040039BB248BF83F010038A063D
S315080012C048BF83F0200343F4004343F080030360E0
S315080012D0704700BF800000F1804000F5B840036801
S315080012E0CA0423F4804323F070039BB248BF83F4F7
S315080012F080538A0448BF83F4005343F4004343F001
S3150800130080030360704700BF800000F1804000F54D
S31508001310B840036823F4E04323F040039BB283F00C
S31508001320300343F4004343F080030360704700BF73
S31508001330800000F1804000F5B840036823F480433C
S3150800134023F070039BB283F4405343F4004343F005
S3150800135080030360704700BF40F60F62800000F10B
S31508001360804000F5B8400368134043F4004343F057
S3150800137080030360704700BFFFF7EEBF800000F1EF
S31508001380804000F5B84003685B0408D540F60F7343
S315080013900268134043F4404343F0800303607047F8
S315080013A0800000F1804000F5B84003685B0608D568
S315080013B040F60F730268134043F4004343F0C0033A
S315080013C003607047044A054B126892B202EBC000EC
S315080013D003445B0019607047505C004002300020EF
S315080013E00E4A0F4B12683E2992B202EBC000034424
S315080013F04FEA43030AD94A09C80604BF02F1FF3275
S3150800140092B2920242F400421A6070474A08C9072B
S3150800141048BF013292021A60704700BF505C004014
S3150800142006300020064B49081B6849009BB203EBAF
S31508001430C00000F1005000F54050400001607047C0
S31508001440505C0040FFF7EEBF054A064B1268490894
S3150800145092B202EBC000034449005B001960704772
S31508001460505C004004300020FFF7EEBF054B1B68B8
S315080014709BB203EBC00000F1005000F5405040005D
S3150800148000887047505C0040FFF7F0BF044A054BE0
S31508001490126892B202EBC00003445B0018887047DA
S315080014A0505C004004300020FFF7F0BF054A064BA9
S315080014B0126892B202EBC00003445B001868C0F3DE
S315080014C009007047505C004006300020FFF7EEBF69
S315080014D0C3B2000A40EA0320704700BF08B538B116
S315080014E0064B1B681B689847054B18680A3008BDE9
S315080014F0034B01221B681A8208BD00BFA0130020F7
S31508001500A413002008B538B1064B1B689B6898479A
S31508001510054B18680C3008BD034B01221B681A825C
S3150800152008BD00BFA0130020A413002008B51F4B58
S31508001530002832D01E481A6800210180137813F05B
S315080015407F0316D0012B27D0022B24D1527902F023
S315080015500F039B0003F1804303F5B84312061B688B
S315080015601FD403F44053B3F5805F0ED101230370F3
S315080015700BE0527A930654BF0378022351064CBFF8
S3150800158043F0010323F0010303700A4B1B681B6930
S315080015909847074808BD084608BD1B6802221A82F4
S315080015A008BD03F03003102BEFD1DFE7A4130020AA
S315080015B0AC130020A01300202DE9F041244F3C680D
S315080015C0258A2DB9267A042E2AD0A38A042603E072
S315080015D0A38A9D42FAD902269D4228BF1D46A369C1
S315080015E02846984780460020FFF74EFF2A460146C0
S315080015F04046FFF7DBFD29460020FFF7E3FE638A36
S31508001600228A1449521B1D44134B228265823020BC
S315080016104FF440523C6808801A802672BDE8F08173
S315080016200E4B1A78012A06D00A4B102207261A8072
S315080016302672BDE8F0810A490A4A0968054889B24E
S315080016400A445200156030223C681D700280E4E7A7
S31508001650A4130020B0130020AE130020200500209C
S31508001660505C0040023000200B4B0C4A1B68517836
S31508001670DA78914201D20220704799780029FAD186
S3150800168010B59C880CB1022010BD05499A720B68EA
S315080016905B689847204610BDA4130020B0000020C0
S315080016A0A013002038B5104A104C12682368D97860
S315080016B058799369984723689A7A0AB9022038BDF7
S315080016C00028FBD11A79002AF8D19D78002DF5D18A
S315080016D0074B1B68DB689847236828465979DA78E8
S315080016E0D9721A7338BD00BF7C130020A4130020DA
S315080016F0A013002038B5314B1B68187810F07F000E
S3150800170003D0022806D0022038BD5A7A22F02002D9
S315080017105A7238BD5A88002AF6D11A79002AF3D1A6
S315080017205A7922F080008400150604F18041244D80
S3150800173001F5B84109682D784CBF01F0300101F474
S315080017404051A842DFD20029DDD09B7A002BDAD09F
S3150800175004F1804404F5B8441206236809D503F059
S315080017603003102B1ED0174B1B685B699847002067
S3150800177038BD03F44053B3F5805FF4D1D8B9124BA2
S3150800178093F82C10FFF72CFE236823F4804323F0EC
S3150800179070039BB283F4405343F4004343F0800341
S315080017A02360E0E7C4B22046FFF7FAFD2046302161
S315080017B0FFF776FDD7E7FFF7E1FDE5E7A41300207D
S315080017C0B0000020A01300202400002038B5224BCA
S315080017D01868427922F080018C00150604F18043CE
S315080017E01E4D03F5B8431B682D784CBF03F0300334
S315080017F003F44053A94201D3022038BD4188002989
S31508001800FAD1002BF8D0837A002BF5D004F1804466
S3150800181004F5B8441206236811D523F4E04323F0EF
S3150800182040039BB283F0100343F4004343F0800364
S3150800183023600B4B1B689B699847002038BD23F42F
S31508001840804323F070039BB283F4805343F4004330
S3150800185043F080032360ECE7A4130020B0000020C7
S31508001860A0130020054B1B685A8A10B1086810445B
S31508001870704789888A1A1A82704700BFA413002005
S3150800188010B50C4B002093F82C10FFF7A9FD0A4B56
S315080018901B68187A082806D10849094B4FF4805462
S315080018A010220C801A80A0F10900B0FA80F04009D5
S315080018B010BD00BF24000020A4130020AE13002092
S315080018C0B013002070B5A24DA24A2B6811681A7A87
S315080018D082B0092A3ED0A04A89B20A445200148826
S315080018E0640004F1804404F5C04422781A702B6819
S315080018F062785A70A0882E68FFF7EAFD7080208902
S315080019002E68FFF7E5FDB080A2892B680121DA80F1
S31508001910197222B35878062800F0848000283AD134
S315080019205988002900F098808C4C23681B699847D1
S31508001930032800F0EA804FF6FF722C68238A934248
S3150800194000F08480022836D108232372FFF798FF17
S3150800195002B070BDDA8801211972002ADAD11A7824
S315080019605C7812F07F0236D0012A00F0BF80022A86
S3150800197000F0E180794B20461B685B69984703288D
S3150800198000F0C38000283ED02B6808221A72FFF7A1
S3150800199077FF02B070BD082870D11A785206C3D1F5
S315080019A06F4A00209A61588290474FF6FF722C685A
S315080019B0238A93424AD0002BC6D094F90020002AE5
S315080019C07FDB684A4FF44051032311802372FFF7E7
S315080019D057FF02B070BD092C00F0E180052C00F01D
S315080019E09B80032C00F0CA80012CC3D1DA78012A27
S315080019F0C0D19A88002ABDD15B7A9B06BAD5FFF773
S31508001A0079FE0028B6D1534A574B1268002192B284
S31508001A1013445B001960554A30212B681180062251
S31508001A201A72B4E71A7856067FF47EAF9A784B4C4A
S31508001A30012A00F0BA80022A6BD0032A7FF475AF18
S31508001A402268526A002AACD106206EE7092323725F
S31508001A50FFF716FF02B070BD5A6822F47F42B2F54E
S31508001A60003F7FF461AF187810F07F0040F0A08047
S31508001A709A88002A7FF458AF3D4A92E70A287FF4ED
S31508001A8053AF1A7802F07F02012A7FF44DAF9A7A93
S31508001A90002A3FF449AF598800297FF445AF5A68B0
S31508001AA02E4C22F47F42B2F5803F7FF43EAF226887
S31508001AB05879936998472B68002840F0B6802D4AD4
S31508001AC06FE7E288019201998B4217D8934276D242
S31508001AD0224A126892F82C108AB2934274D2264B84
S31508001AE000211970A282FFF767FD70E70B2C7FF4BF
S31508001AF041AFFFF7D7FD002885D03BE7174B019A82
S31508001B001B68228293F82C20ECE72B6809221A72AC
S31508001B103DE72268126A95E793F90320002A07DB56
S31508001B209A782AB99A881AB99A7A002A3FF46BAF32
S31508001B3008221A722BE7012C3FF461AF032C7FF4BD
S31508001B4019AFFFF743FE00283FF45DAF12E700BF69
S31508001B50A4130020505C0040043000207C130020B1
S31508001B60DD140008AE13002002300020B013002058
S31508001B702D1500080515000820050020DA78012A29
S31508001B807FF4F8AE9A88002A7FF4F4AE5A7A284988
S31508001B9042F0200209685A72CB69984733E7FFF783
S31508001BA063FD00283FF42FAFE4E62268D26949E7CF
S31508001BB001282FD0022811D008461E4CB5E61D4B29
S31508001BC01B6893F82C208DE793FBF1F001FB10338B
S31508001BD0002B87D1184B0121197083E7587900F03B
S31508001BE00F018A00040602F18042144C02F5B8423D
S31508001BF0126824784CBF02F0300202F44052A14227
S31508001C0006D210F0700003D1002A7FF435AF8BE6B8
S31508001C10002089E6074C58792268936998472B680B
S31508001C2018B99A7A002A7FF427AF58787DE600BF5C
S31508001C30A01300207C13002020050020B0000020FF
S31508001C40F8B5304D2C68237A022B07D0042B05D023
S31508001C50032B09D0052B07D0072B33D00823237273
S31508001C60BDE8F840FFF70CBEA369228AB3B1B2B14A
S31508001C70A68A964228BF164630469847228A638A1D
S31508001C80921B33440746228263820020FFF70CFC2E
S31508001C90324601463846FFF79DFA228ACAB9A38A10
S31508001CA033B319492A68194B062010721A68184B5B
S31508001CB092B213445B0000221A602C683022237A01
S31508001CC00A80CCE7134B1B68DB6898472C68082307
S31508001CD0C5E7114B00214FF4405208461A80FFF71A
S31508001CE071FB238AA28A084930209A42088003D8C1
S31508001CF02C6803232372B2E7002BD3D02C68052364
S31508001D002372ACE7A4130020B0130020505C0040F7
S31508001D10023000207C130020AE130020F8B5234CB7
S31508001D2023681A7A022A17D0042A15D0062A05D05B
S31508001D3008221A72BDE8F840FFF7A2BD5A78052AAC
S31508001D4013D01B4B1B689B689847236808221A7296
S31508001D50BDE8F840FFF794BDFFF72EFC23681A7A12
S31508001D601A72BDE8F840FFF78BBD1A7812F07F02A9
S31508001D70E7D11049DF780E7876B10F4840F60F7133
S31508001D80056842F40043294043F0800301320B43BF
S31508001D90964240F8043BF1D1084A47F08007084BC1
S31508001DA017601B681B6A9847CBE700BFA41300207F
S31508001DB07C130020B0000020005C00404C5C004012
S31508001DC0A013002070B40C4B1E787EB10B4C002279
S31508001DD040F60F71256842F40043294043F080031A
S31508001DE001320B43964244F8043BF1D1044B40F0D0
S31508001DF08000186070BC7047B0000020005C00408E
S31508001E004C5C0040704700BF2DE9F04FDFF87CA11D
S31508001E10DFF87C915746C84685B00023DFF874B1D1
S31508001E20554DADF80E30DBF80030544C99B21B0412
S31508001E30534E514AAAF8001040F191803B8803F0AE
S31508001E400F03990001F1804101F5B84189F8003086
S31508001E50002B2FD14BF6BF73216889B229802988B8
S31508001E6001F030013180298801F440512980216828
S31508001E700B4083F4005383F0200343F4004343F0FC
S31508001E80800323603B88D90641D523689BB2ADF809
S31508001E900E30BDF80E301B0564D4BDF80E3018049C
S31508001EA0C1D540F68F73019221680B402360FFF776
S31508001EB0C7FE34E00B689BB2ADF80E30BDF80E30A5
S31508001EC0180417D4BDF80E301A06ACD548F60F72AA
S31508001ED099F800302B499B0003F1804303F5B8437A
S31508001EE0186802401A6099F80030013B51F823300F
S31508001EF0984798E740F68F730868234A03400B60B3
S31508001F0098F80030013B52F823309847DAE748F64C
S31508001F100F73019221680B402360FFF7FFFE4BF613
S31508001F20BF73019A2068118812880340C90448BF04
S31508001F3083F480539704328848BF83F40053D50648
S31508001F40328848BF83F01003940648BF83F0200305
S31508001F5043F4004343F08003084A9BB2136005B07C
S31508001F60BDE8F08F40F68F73019221680B4023601D
S31508001F70FFF7A8FCD3E700BFAE130020005C0040C3
S31508001F80B0130020B4000020D000002074130020F5
S31508001F9080130020445C004038B50120FEF7F4FAAF
S31508001FA0064D074B074C00224FF4E05101201860FC
S31508001FB01A602A6021801960104638BD445C0040CA
S31508001FC0405C0040A8130020054B00221A709A6452
S31508001FD083F84220A3F844209A705A70704700BFCD
S31508001FE028050020024B1878003018BF01207047DA
S31508001FF028050020024B002283F84220704700BFC4
S315080020002805002070B50578FF2D41D0B44C2378FB
S31508002010012B00D070BDC93D0646352D00F246811C
S31508002020DFE815F000014401440191004401440130
S3150800203099007D00A100AE00440144014401440119
S31508002040440144014401440144014401440144015A
S31508002050440144014401440144014401440144014A
S31508002060440144014401440144014401440144013A
S315080020704401440144014401BD00D5003001170163
S315080020804401440144011F014401E200EA00F7004B
S3150800209000F036FA924CE8B9FE2110220223E170CC
S315080020A02271A4F8443094F842308D4A012B09D0A5
S315080020B0B2F84410012384F842308A48BDE87040DB
S315080020C000F038B9FE2210230221E2702371A4F829
S315080020D04410EFE700231022012663706371227112
S315080020E0E570267000F046F9A07100F035F9E07148
S315080020F000F032F90823D84020726672A672A4F856
S31508002100443000F04BFD94F84230754A012BD9D083
S31508002110B2F9441000297FF77DAF89B2CAE700F00B
S3150800212029F973780138984256DDFF220123E270B7
S31508002130A4F8443071786A4D002940F0C48000F054
S3150800214037FD0028DFD1FE2131220223E1702271FA
S31508002150A4F84430A7E700F0D1FEFF220123E2707D
S31508002160A4F844309FE74168A06C5D4D00F01AFD65
S315080021700028E8D0FF220123EA70A5F8443092E748
S315080021800025FF23E3702571657100F0F3F8072336
S31508002190A071E57125726572A4F8443083E7FF23C0
S315080021A0E3704368A26C3BB1D018002312F8011BF8
S315080021B00B448242DBB2F9D1002201200821C4F87F
S315080021C0073020716271A271A4F844106BE700F021
S315080021D0D1F87378984271DCFE2122220223E1703D
S315080021E02271A4F844305EE7FE2100220223E17042
S315080021F02271A4F8443056E760780023FF210622AE
S315080022006071E1702371A371E3712372A4F844200D
S3150800221049E70023FF21012223706370E170A4F8C7
S31508002220442040E7A56C00F0A5F8721C411E28461C
S315080022302B4D00F0B5FC002885D0FF23EB7000F08D
S3150800224099F8AB6C013803440122AB64A5F8442025
S3150800225029E7FF23E37042680123A264A4F8443007
S3150800226021E7214D0023FF2007210822A564E070FD
S3150800227023716371A37123726372A372E171A4F867
S31508002280442010E700F076F872789042A4DDA16C3D
S31508002290164800F053FEFF23E3707378A26C1344CC
S315080022A0A36473780133A4F844302CE7FE21202276
S315080022B00223E1702271A4F84430F4E671680B48F1
S315080022C0A1647278E5E7B21CA86C00F069FC0028E6
S315080022D03FF439AF7378AA6C1344AB6413E700BFB5
S315080022E0280500202B0500208C5400082C0500200A
S315080022F008B5FFF769FE00F0D1FC024B02221A70FE
S3150800230008BD00BFED00002008B5074800F02CFD09
S31508002310012800D008BD054B02221A700248BDE804
S315080023200840FFF76FBE00BF74050020ED000020CF
S3150800233000F0E6BC08B5074B1B78022B03D0BDE8B6
S315080023400840FFF757BEC9B200F0DEFCBDE80840FA
S31508002350FFF750BEED000020044B1B78032B9ABFF5
S31508002360034A32F813003F20704700BFED000020F3
S3150800237094540008FFF7F0BFFFF734BE10B5FFF717
S31508002380FBFF012806D000F0BBF818B10B4C2378E8
S31508002390012B00D010BD01F047F8094B1B6803F567
S315080023A0FA639842F6D30023237000F0B1F80028A8
S315080023B0F0D1BDE8104000F0A1BD00BFB305002074
S315080023C0B405002008B5054B01221A7001F02CF857
S315080023D0034B1860BDE80840FFF7D0BFB3050020DF
S315080023E0B405002008B500F087FD00F01BF800F0E2
S315080023F0F3FF00F0D3FB00F069F8FFF779FFBDE8BB
S315080024000840FFF7DFBF00BF08B500F00DF800F081
S31508002410FDFF00F07FF9FFF777FFBDE80840FFF7FB
S31508002420ADBF00BFFEF7ECB8FEF7EEB8092800F01E
S315080024300F0302D903F13700704710B503F13004D2
S3150800244002F076FF2044437803F00303022B14BFFF
S315080024502046A4F12000C0B210BD00BF38B505461D
S3150800246000090C46FFF7E2FF207005F00F00FFF7A2
S31508002470DDFF00236070A370204638BDF8B500263E
S31508002480471E451C17F8014F02F052FF20444378B7
S3150800249003F00303022B08BF203CE3B2A3F130028A
S315080024A0D2B2162AA3F13A010DD806290BD9092A60
S315080024B084BF373BDAB202EB0613AF4203F0FF06DE
S315080024C0E0D13046F8BD0020F8BD00BF10B50023A6
S315080024D0074C1A4607490848237002F0E3F900B981
S315080024E010BD77210548BDE8104000F053BB00BF7A
S315080024F0F80500209C54000804060020A054000893
S31508002500024B1878B0FA80F040097047F8050020A9
S3150800251010B5FFF731FF012802D0054C23780BB11F
S31508002520002010BDFEF772F80128F9D1207010BD01
S31508002530F805002038B50546047802F0F9FE20446F
S31508002540437803F00303022B08BF203C532C01D029
S31508002550032038BD02F0ECFE6B7818444278520727
S31508002560F6D5312B05D0322B05D0332BF0D10220EE
S3150800257038BD002038BD012038BD00BF70B50646FD
S315080025800230FFF77BFF0546043684B23046FFF774
S3150800259075FF013CA4B22844012CC5B206F1020617
S315080025A0F4D83046ED43FFF769FFEDB2281AB0FAC2
S315080025B080F0400970BD00BF2DE9F041044616467B
S315080025C00F46002949D0002847D02046FFF7B2FF1A
S315080025D0032805463ED02046FFF7D0FF002800F026
S315080025E09280012D3FD06BD3022D33D1A01CFFF76B
S315080025F045FF0546201DFFF741FF00063860A01D70
S31508002600FFF73CFF3B6804F10C0803EB0040386019
S3150800261004F10800FFF732FF3B6803EB002038603F
S3150800262004F10A00FFF72AFF3B686C1F184424B21E
S31508002630386066B1002C0ADD00254046FFF71EFF0C
S315080026406B1C70559DB2A54208F10208F5DB2046C1
S31508002650BDE8F0810020BDE8F08140F261212C48F8
S3150800266000F098FAB1E7A01CFFF708FF0546201D01
S31508002670FFF704FF00043860A01DFFF7FFFE3B6864
S3150800268004F10A0803EB0020386004F10800FFF79C
S31508002690F5FE3B682C1F184424B23860002ED6D0AD
S315080026A0002CD4DD00254046FFF7E8FE6B1C70556C
S315080026B09DB2A54208F10208F5DB2046BDE8F08187
S315080026C0A01CFFF7DBFE0546201DFFF7D7FE00021C
S315080026D03860A01DFFF7D2FE3B68033D18442DB2B3
S315080026E00834386066B1002D0ADD00272046FFF75A
S315080026F0C5FE7B1CF0559FB2AF4204F10204F5DB20
S315080027002846BDE8F0814FF0FF30BDE8F08100BFF4
S31508002710A05400082DE9F843AA4F3C783CB1012C97
S3150800272000F01781022C00F08E80032C01D0BDE842
S31508002730F883A54EA54D06F50C7228464FF4807110
S3150800274002F0EAFC96F84192B9F1000F40F0BB811D
S31508002750002855D005F5807205F5C0712846FFF7A3
S315080027602BFFB0F1FF3F804600F01E81002847DDB1
S315080027709748FDF7A1FF43469649974AA2FB0303EC
S31508002780DB0801F10101F9D1444693480B70A0FB1F
S315080027900423DB0803EB8302A4EB4202303201F880
S315080027A0012D1C46002BF2D18A48FDF785FF8B4880
S315080027B0FDF782FF874995F88301FFF74FFE8849A1
S315080027C095F88201FFF74AFE864995F88101FFF7D9
S315080027D045FE854995F88001FFF740FE7D48FDF7DF
S315080027E06BFF8248FDF768FF4146D5F88001804AAD
S315080027F000F0D6F9002800F079817E48FDF75CFFE5
S31508002800D6F84422D6F83C329A4290D17A48FDF757
S3150800281053FF00F0CDF90446002800F08081754882
S31508002820FDF74AFF7548FDF747FF754802F026FB96
S315080028307448FDF741FF00233B70FDF71DFFBDE817
S31508002840F84300F05BBB604E604D06F50C722846F7
S315080028504FF4807102F060FC96F84192B9F1000FCE
S3150800286040F03F81D0B14A4605F5C0712846FFF7CA
S31508002870A3FEB0F1FF3F804600F05D8100280DDD24
S31508002880614C6368002B00F019812268D5F8801125
S315080028901A44914240F0CA8003446360D6F8442241
S315080028A0D6F83C329A427FF442AF0021544802F0EF
S315080028B0F7FA002840F04D81534C6368002B41D04D
S315080028C04C48FDF7F9FE5148FDF7F6FE63684149A5
S315080028D01A464148A0FB0252D20801F10101F9D17A
S315080028E03D4D0A70A5FB0302D20802EB8200A3EB5A
S315080028F04003303301F8013D1346002AF2D135482A
S31508002900FDF7DAFE4248FDF7D7FE3249E078FFF7D1
S31508002910A5FD3349A078FFF7A1FD32496078FFF796
S315080029209DFD31492078FFF799FD2A48FDF7C4FE39
S315080029302E48FDF7C1FE94E8030000F033F900289D
S3150800294000F0E0802B48FDF7B7FE03233B70BDE897
S31508002950F88300F023F9FDF77BFE2E48FDF7ACFE61
S315080029602D48FDF7A9FEFDF76FFE224601462448CD
S3150800297001F0CAFF054638B12848FDF79DFE2046F6
S31508002980BDE8F843FDF78EBE1A48FDF795FE2448C4
S31508002990FDF792FE2348FDF78FFE1B4B02221D60B2
S315080029A05D603A70BDE8F8831F48FDF785FE20464E
S315080029B0FDF778FE06F50C7002F060FA87F80090CD
S315080029C0BDE8F883F8050020040600205C0A00200C
S315080029D0D8550008B8050020CDCCCCCCE855000861
S315080029E0BA050020BC050020BE05002018560008C0
S315080029F05C0B00200C550008005600081C56000801
S31508002A003408002034560008FC05002068550008E4
S31508002A1074550008B8540008DC540008045500082A
S31508002A201455000838550008B45500084B48FDF7FA
S31508002A3043FE4B48FDF740FE63684A491A464A4832
S31508002A40A0FB02E2D20801F10101F9D1DFF818E191
S31508002A500A70AEFB0302D20802EB8200A3EB400326
S31508002A60303301F8013D1346002AF2D13D48FDF7FF
S31508002A7023FE3E48FDF720FE3A49E078FFF7EEFCD4
S31508002A803B49A078FFF7EAFC3A496078FFF7E6FC8D
S31508002A9039492078FFF7E2FC3248FDF70DFE374842
S31508002AA0FDF70AFE94E80300354C00F07BF848B3BE
S31508002AB02A48FDF701FE3348FDF7FEFDD5F88031BB
S31508002AC084E80801EAE63048FDF7F6FD0220FDF73E
S31508002AD0E9FD06F50C7002F0D1F900233B70BDE85C
S31508002AE0F8832A48FDF7E8FD2046F0E72748FDF772
S31508002AF0E3FD0620FDF7D6FD254802F0BFF93C7038
S31508002B00BDE8F8832148FDF7D7FD0520FDF7CAFD86
S31508002B101F4802F0B3F900233B70BDE8F8831B4851
S31508002B20FDF7CAFD0720FDF7BDFD194802F0A6F915
S31508002B303C70BDE8F8831548FDF7BEFD0320FDF798
S31508002B40B1FD06F50C7002F099F987F80090BDE81A
S31508002B50F8830E48FDF7B0FD0420D7E70C550008AA
S31508002B6068550008B8050020CDCCCCCC74550008B3
S31508002B70BA050020BC050020BE050020185600082E
S31508002B80FC05002038550008905500080455000833
S31508002B903408002008B5FFF747FCFCE700F0DCBA6C
S31508002BA000F0DCBA00F004BB00F0D0BB00F010BCAB
S31508002BB008B500F0A7FB00B908BDBDE8084000F05D
S31508002BC0EDBB00BFB2B1002370B41E46541EE4B27A
S31508002BD001346400020F092A02F1300586BF373234
S31508002BE0CA54CD54CA180233A3424FEA001056708D
S31508002BF0F0D170BC704700BF012838B504460D46B1
S31508002C0004D94FF4FC710F48FFF7C4FF04EB4404E2
S31508002C100D48E4000319597C1A7C914210D0DA68F1
S31508002C201570DA68597C5D6801320131AA42597417
S31508002C30DA6003D902590120DA6038BD012038BDAF
S31508002C40002038BD60560008680C0020012870B5C1
S31508002C5004460E4604D940F21A210E48FFF79AFF99
S31508002C6004EB44040C4DE4002B19587C80B19A6897
S31508002C70127832709A68597C586801320139824252
S31508002C8059749A6003D92A5901209A6070BD0120A7
S31508002C9070BD00BF60560008680C0020F0B4144BE5
S31508002CA0144C1549651C04F14000144F03F1180231
S31508002CB001F140065A6158600022481CDE619D6099
S31508002CC00126DD601D6040259A74DA625A7483F81D
S31508002CD029203A601862586298610E7083F82A6053
S31508002CE01D7483F828502270F0BCFEF783BA00BF23
S31508002CF0680C00201C0D0020980C0020640C002095
S31508002D000020FDF741BC00BF3F2970B50D460446BB
S31508002D1021D8134E29463078FFF76EFF012803D0D5
S31508002D209D211048FFF736FFADB29DB1013DADB20A
S31508002D302544013CFFF778FB14F8011F3078FFF7AC
S31508002D405BFF01284FF0A601064801D0FFF722FFD6
S31508002D50AC42EFD170BD99210248FFF71BFFD8E7B7
S31508002D601C0D002060560008F8B5194D0646FDF7FB
S31508002D70EBFC2C7854B9174B174E18783146FFF7E9
S31508002D8065FF01281CD000242046F8BD134C114BC2
S31508002D902178114F013139441878FFF757FF012878
S31508002DA0F1D123783A780133DBB29A422370EAD11B
S31508002DB00446791C304600F0C1F800232B70E3E77F
S31508002DC03378002BDFD0054B28701C70DCE700BF7A
S31508002DD0200C0020980C0020E00B00205D0D002040
S31508002DE0F0B51D4F83B03C78012C04D940F23A2146
S31508002DF01A48FFF7CFFE1A4B04EB440403EBC4044E
S31508002E00667C3EB3402E174D28BF402600240DF1A0
S31508002E1007013878FFF71AFF012804F101040F4863
S31508002E2003D040F24911FFF7B5FE9DF80720E3B23B
S31508002E309E4205F8012FEAD8B6B232464FF48071A1
S31508002E400948FEF7B3F901203146FEF7BBFA01201F
S31508002E50FEF75AFA03B0F0BD1C0D002060560008B4
S31508002E60680C0020230C0020240C002070B50F4CA1
S31508002E7001202146FEF7ECF980B290B1451EADB2AD
S31508002E800B4E2544013C14F8011F3078FFF7B4FEB9
S31508002E9001284FF4B771074801D0FFF77BFEAC4213
S31508002EA0F1D10120BDE87040FEF742BADC0C0020E3
S31508002EB0980C00206056000810B50A4B0A490B4AC0
S31508002EC01B680C681068181800D110BD082208493C
S31508002ED0FFF778FE2046BDE8104004220549FFF7B3
S31508002EE071BE00BFE8F7FF1FECF7FF1FF0F7FF1FE3
S31508002EF0020000201200002000F0A4BA10B5FFF767
S31508002F0053FE00B910BDFDF76FFB0028FAD0FFF796
S31508002F100FFA00F075FAFFF749FE074B20F06040FC
S31508002F2020F07F001860FFF741FE446800F08CFA35
S31508002F302346BDE81040184708ED00E072B170B5A9
S31508002F400D46561EB6B20644441E15F8013B04F853
S31508002F50013FFFF769FAB442F7D170BD704700BF69
S31508002F602DE9F041DFF83C80074646460C4D002423
S31508002F7001E056F80C5FFFF757FABD4203D87368AD
S31508002F801D44AF4205D301340D2CF2D1FF20BDE814
S31508002F90F08104EB440408EB8404207ABDE8F08150
S31508002FA000600008885600082DE9F04107460068C9
S31508002FB0FFF7D6FFFF2845D0244A2548254934235C
S31508002FC050605160D360D36813F0010327D11446CB
S31508002FD0116941F00101116103F1040857F808600D
S31508002FE03D68B2B25A53E2681D44D00704D5FFF7CC
S31508002FF01BFAE368DA07FAD4330C6B80E368D9075F
S3150800300004D5FFF711FAE368DB07FAD42B689E426A
S315080030100CD1B8F5007F4346DED1012007E01369DD
S31508003020002043F080031361BDE8F0810020074BC0
S315080030301A6922F001021A611A6942F080021A61BD
S31508003040BDE8F0810020BDE8F08100BF0020024005
S3150800305023016745AB89EFCD38B5104B0D4698422D
S3150800306019D00F4A914208D00446FFF79DFF10B1C8
S31508003070C5F3080313B1002038BD1C462368AB42CC
S3150800308007D02046294640F8045B4FF40072FFF744
S3150800309055FF204638BD034CEAE700BF600D002007
S315080030A000600008640F00202DE9F8430C4601680B
S315080030B024F4FF781D464B1C0746164628F00108DF
S315080030C032D0884506D038464146FFF7C5FF074641
S315080030D038B30168641A3C44043408F5007807F1EB
S315080030E0040905E016F8013B013D04F8013B15D03B
S315080030F0FFF79AF9C9EB0403B3F5007FF2D3384614
S315080031004146FFF7A9FF074600F1040948B14C46B6
S3150800311016F8013B013D04F8013BE9D10120BDE861
S31508003120F8830020BDE8F883814649F8048B4146B8
S3150800313048464FF40072FFF701FF3968C1E700BF40
S315080031400349044A4FF0FF330B601360704700BF12
S31508003150640F0020600D0020FFF7F2BF70B50D4622
S3150800316016460446FFF7FCFEFF2814D0681E2044C6
S31508003170FFF7F6FEFF280ED00A4A24F4FF7323F061
S315080031800103934221462B46324606D0BDE87040DD
S315080031900548FFF789BF002070BD0448BDE87040A8
S315080031A0FFF782BF00600008640F0020600D002052
S315080031B02DE9F0470C460646FFF7D2FE0546601E87
S315080031C03044FFF7CDFE85426BD8EB1EDBB2FB2BF6
S315080031D067D80F28044664D8464A474847493423DF
S315080031E050605160D360D36813F0010668D1136943
S315080031F0434F43F00203B846B94613614FF0030A3A
S3150800320001E099F808A0FFF70FF9554509F10C09EF
S315080032105DD001360D2EF4D14FF0FF36DFF8E09081
S3150800322000254FF0030A01E099F808A0FFF7FCF81B
S31508003230544509F10C0957D001350D2DF4D14FF03D
S31508003240FF3900254FF0030A01E097F808A0FFF7B9
S31508003250EBF8544507F10C073FD001350D2DF4D195
S315080032600023C6EB09094B44C3F38F23E3B15F1E62
S31508003270BFB206F580651F4C05EB87276661236993
S3150800328043F040032361E368DA0704D5FFF7CCF877
S31508003290E368DB07FAD4AF422E4605D005F580650C
S315080032A0ECE70020BDE8F087124B01201A6922F0EE
S315080032B002021A611A6942F080021A61BDE8F087B3
S315080032C01369002043F080031361BDE8F087F6B266
S315080032D006EB460658F82660A0E7EDB205EB45056D
S315080032E008EB85056B68BCE7EDB205EB450558F8B4
S315080032F02590A6E70020024023016745AB89EFCD5C
S31508003300885600080F4B1A68013218D030B59968EC
S315080033105C68DD6818690C442C445969044498694A
S315080033200C44D969231883B00B4402AA5B4242F8BD
S31508003330043D04210448FFF711FF03B030BD012006
S31508003340704700BF600D0020EC60000810B40E49FD
S315080033500E4B0F4A08681B680E4C12680C31034462
S3150800336009680D48134422680B4401681344A2688F
S315080033700B44D0F8D8101344CB4200F1D80010BC47
S315080033800CBF012000207047006000080460000898
S3150800339008600008106000081460000808B50A48AC
S315080033A00368013302D0FFF7FFFD58B107480368E9
S315080033B0013305D0FFF7F8FD003018BF012008BD1E
S315080033C0012008BD08BD00BF600D0020640F002065
S315080033D0004870470060000810B4064B064C0749C1
S315080033E0002205201A605C609A6018600A6010BCAA
S315080033F0704700BF10E000E03F1901006811002087
S31508003400014B00221A60704710E000E0044B1B686D
S31508003410DB0303D5034A136801331360704700BF03
S3150800342010E000E068110020044B1B6813F4803F8D
S31508003430034B18681CBF01301860704710E000E0A5
S315080034406811002072B6704762B670470168F1B11C
S3150800345010B40C781F2C09D93A2C14D00A4601E06E
S315080034603A2B06D012F8013F1F2BF9D8002010BCC2
S31508003470704701318A4206D1302C04D101320260EC
S3150800348010BC002070474FF0FF3010BC70474FF05B
S31508003490FF30704758B110B5036882B004460BB1C7
S315080034A01A7842B900230B60092002B010BD002328
S315080034B00B6009207047D888A2889042F2D15878C4
S315080034C00191FDF7CBFB10F001000199EAD12368C1
S315080034D00B60EAE701380A4411F8013B914200F80B
S315080034E0013FF9D1704700BFF8B5C46A00F130074B
S315080034F005462246394640780123FDF70BFCB0B94C
S315080035002A6AAB69A21A9A42E8700ED2AE78012EE0
S3150800351001D80AE0AB691C44013E2246012339461C
S315080035206878FDF7F7FB012EF4D10020F8BD0120DD
S31508003530F8BD00BF38B5C36A8B4218D0C3780446B5
S315080035400D467BB92A46012304F130016078FDF760
S315080035508FFB002818BF4FF0FF35E5620CBF00202F
S31508003560012038BDFFF7C0FF0028EBD038BD00208A
S3150800357038BD00BFF8B5C37805465BB92B78032B71
S315080035800DD0002268781146FDF72AFC003018BFD6
S315080035900120F8BDFFF7A8FF0028EFD0F8BD2B796A
S315080035A0012BEED105F130010B4605F50C70002212
S315080035B003F8012B83424FF00004F9D12B69E86820
S315080035C01F0A1E0CEA6985F818321B0E4FEA102EE0
S315080035D085F8197285F81A62070C060E85F81B32EB
S315080035E085F81C02AA235520013285F81E7285F833
S315080035F01F625227612685F82E0285F82F32412050
S31508003600722385F8330085F8160285F8143285F892
S31508003610153285F81DE2EA6285F8307085F8317052
S3150800362085F8326085F8176201236878FDF772FB22
S315080036302C71A6E700224FF0FF3310B5C270C362A3
S315080036400446FFF777FF08B1042010BD4AF6552255
S3150800365094F82F1294F82E3243EA0123934201D0AC
S31508003660032010BDB4F8681094F8673094F8662003
S3150800367043EA012342EA03230A4923F07F438B42A4
S31508003680EFD0B4F8840094F8833094F8822043EAA3
S31508003690002342EA032323F07F438B4214BF022010
S315080036A0002010BD46415400F0B5002385B00B60DC
S315080036B00F461446FFF7CAFE061E18DBC34B53F81F
S315080036C02650BDB13D602B7804F0FE0423B168781E
S315080036D0FDF7C4FAC70710D5F0B2002368702B703F
S315080036E0FDF754F9C60711D5032005B0F0BD0B2028
S315080036F005B0F0BD0C2005B0F0BDCCB300F0040356
S3150800370003F0FF00002BF0D00A20EEE70CB14107CA
S31508003710FAD400212846FFF78DFF022806D0042890
S3150800372024D0012840F2CE800D20DEE76C4668469C
S3150800373005F5FC7305F50E7613F8062C42B11F88BD
S3150800374013F8012C13F8021C42EA072241EA022266
S315080037501033B34240F8042BEED104AF54F8046B8F
S3150800376003203EB9A742F9D10428DDD10120BCE7E0
S315080037702046BAE731462846FFF75CFF0128F1D80C
S3150800378095F83C2095F83B3043EA0223B3F5007FD1
S31508003790CAD195F8471095F8463053EA012340F008
S315080037A09380B5F8561095F8553095F8542043EAA5
S315080037B0012342EA032195F84070A9617B1E012B7B
S315080037C0AF70B1D895F83D309AB26A81002AABD06D
S315080037D05A1E1A42A8D195F8412095F8424042EA65
S315080037E0042422072C819FD195F8440095F843209C
S315080037F052EA002209D1B5F852E095F8510095F839
S31508003800502040EA0E2042EA002295F83FE095F85B
S315080038103E0050EA0E2087D001FB07F700EB141E86
S31508003820BE44724580D3CEEB0202B2FBF3F3002B03
S315080038303FF47AAF40F6F572934240F2A5804FF610
S31508003840F572934240F2848095F85B7095F85A2099
S3150800385002333044B64452EA07226B612862C5F83F
S3150800386028E0EE617FF460AF002C7FF45DAFB5F819
S315080038705E4095F85D0095F85C209B0040EA0420C0
S3150800388003F2FF1342EA0022B1EB532F6A62FFF4F8
S315080038904BAF95F8611095F860304FF0FF3243EA68
S315080038A00123012B4FF080012A61EA6029710DD0AE
S315080038B00323474A2B701388002001339BB21380D9
S315080038C0EB8012E700265BE7194674E7711C284669
S315080038D0FFF730FE0028EBD14AF6552295F82F025D
S315080038E095F82E32002143EA002393422971DFD14D
S315080038F0698E95F8312095F8303042EA012235492B
S3150800390043EA02238B42D3D1B5F8161295F815224D
S3150800391095F8143242EA01222F4943EA02238B42E0
S31508003920C6D1B5F81A6295F81902B5F81E4295F887
S315080039301D1295F8182295F81C3240EA062041EA2D
S31508003940042142EA002243EA01232A61EB60AFE739
S31508003950023330440EEB06026B612862AA62EE61FE
S31508003960002C3FF4E1AE5B0003F2FF133844B1EBE1
S31508003970532F6862FFF4D8AE4FF0FF3380222B61D5
S31508003980EB602A71022394E7023330440EEB0602F9
S315080039906B612862AA62EE61002C3FF4C5AE03F0A3
S315080039A0010202F2FF1203EB430302EB530338440E
S315080039B0B1EB532F6862FFF4B7AE4FF0FF338022A6
S315080039C02B61EB602A71012373E700BF7013002097
S315080039D06C1300205252614172724161012919D952
S315080039E0F8B54269914208D202780646022A0C4680
S315080039F02BD0032A10D0012A01D00120F8BD016A74
S31508003A0004EB540501EB5521FFF794FD78B34FF00D
S31508003A10FF30F8BD01207047016A01EBD411FFF7AA
S31508003A2089FD0028F3D1A10001F4FE7101F13003EC
S31508003A30334458885A78314491F8303042EA0020A5
S31508003A4043EA002020F07040F8BD016A01EB14211A
S31508003A50FFF770FD0028DAD1610001F4FF717318D1
S31508003A6093F8310093F8303043EA0020F8BD316A04
S31508003A70C5F308036F1C334401EB5721304693F80E
S31508003A803050FFF757FD0028C1D1C7F30803334468
S31508003A9093F83000E30745EA00204CBF0009C0F35D
S31508003AA00B00F8BDB1F5001F01D3022070472DE9C0
S31508003AB0F04111F01F080C4602D00220BDE8F08143
S31508003AC0816805460461076829B93B78022B1AD92B
S31508003AD07B6AC3B119467E897602B4422AD3A41BEF
S31508003AE0384608E00128E8D97B699842E5D2A6421B
S31508003AF021D82868A41BFFF771FF431C0146F1D1A2
S31508003B000120BDE8F0813B89B3EB541FD5D9D7F81E
S31508003B102480C5F818806961B8F1000FCDD0C4F3C8
S31508003B200803303708EB54241F44EF61AC610020CA
S31508003B30BDE8F0817B69023B8A1E9A4204D2B7F837
S31508003B400A80BB6A02FB0838C5F81880E3E700BF9D
S31508003B502DE9F04790F800900446B9F1020F0D469A
S31508003B60164657D0B9F1030F2FD0B9F1010F03D07C
S31508003B7002273846BDE8F087016A05EB550801EBD0
S31508003B805821FFF7D7FC07460028F2D108F1010AA9
S31508003B90EB07C8F30808A04453D598F830302046F8
S31508003BA003F00F0343EA061388F83030216A84F8D5
S31508003BB0039001EB5A21FFF7BDFC00284CD1CAF34C
S31508003BC0080AA244C6F3071652E0016A01EBD511AA
S31508003BD0FFF7B0FC07460028CBD1AD0005F4FE750B
S31508003BE005F1300323445A8826F07046120402F081
S31508003BF070421643300C25444FEA162E310E012228
S31508003C0085F83060987083F801E0D970E27038461C
S31508003C10BDE8F087016A01EB1521FFF78BFC074623
S31508003C200028A6D16D0005F4FF756119C6F30722B1
S31508003C30012381F8306081F83120E3703846BDE809
S31508003C40F08788F83060216A84F8039001EB5A21DE
S31508003C502046FFF76FFC08B107468AE7CAF3080A49
S31508003C60A2449AF83020C6F3032622F00F02164320
S31508003C7001238AF83060E3707BE700BF2DE9F04145
S31508003C8007468846066839BBF5687369EDB90125A4
S31508003C902C4606E0012815D001302BD0AC4218D0AE
S31508003CA0736901349C4202D3012D12D9022421469C
S31508003CB03868FFF793FE0028ECD1012C02D9736906
S31508003CC09C421BD30120BDE8F0819D4228BF0125F7
S31508003CD0DEE70020BDE8F0813046FFF77FFE0128C9
S31508003CE0F0D9431C06D073699842ECD34546CFE712
S31508003CF00128E7D14FF0FF30BDE8F0814FF0FF32E1
S31508003D0021463046FFF724FF0028F1D1B8F1000F0D
S31508003D100CD0B8F1010FD5D973699845D2D241466E
S31508003D2022463046FFF714FF0028E1D1726933694D
S31508003D30023A9342F46001D2013B3361337920465B
S31508003D4043F001033371BDE8F08100BF83690BB905
S31508003D50042070472DE9F04F056983B02035B5F585
S31508003D60001F03D3042003B0BDE8F08FC5F308078E
S31508003D700E460446026827BB41690133836131B3A5
S31508003D805389013B13EA55281BD110460192FFF7C8
S31508003D9025FE01288146019A21D9B0F1FF3F32D08C
S31508003DA0536998421DD2861EC4F814905369023B83
S31508003DB09E4204D2B2F80A80936A06FB0838C4F811
S31508003DC0188030371744E76125610020CBE713894F
S31508003DD0B3EB551FF5D80023A3610420C3E70220DF
S31508003DE0C1E7002EF7D0616920460192FFF746FF2A
S31508003DF0019A814648B90720B5E710460192FFF7B0
S31508003E0073FB019A48B10120ADE70128E7D0B0F16C
S31508003E10FF3FF8D0D378002BEFD102F1300302F53B
S31508003E200C70002103F8011B8342FBD15369A9F1E9
S31508003E300206023B9E4238BF936A51892CBF002373
S31508003E4006FB01334FF0000AD3624FF0010B0EE078
S31508003E5082F803B010460192FFF746FB0028D2D13C
S31508003E60019A0AF1010AD36A51890133D3628A4554
S31508003E70EED3D36ACAEB0303D36295E72DE9F04183
S31508003E80416A04464B1C0568066904D0FFF70AFE1A
S31508003E9008B1BDE8F0814FF0E50801270BE0E369BA
S31508003EA083F80080EF7023699E42F2D901462046C6
S31508003EB0FFF74CFF28B9A1692846FFF73BFB002806
S31508003EC0EDD0042808BF0220BDE8F0812DE9F04FA7
S31508003ED0002185B00746D0F80080FFF7E3FD0028EB
S31508003EE04FD14FF0FF334FF0FF0A994656467B6293
S31508003EF00AE00F2B48D0C7F82490FF260021384641
S31508003F00FFF724FF00283CD1B9694046FFF712FBAA
S31508003F10002836D1FC692578002D00F08880E27AE1
S31508003F20E52D02F03F03BB71E5D01207E1D40F2B54
S31508003F302AD076B9214604F10B0011F8013BF201AB
S31508003F4042EA56061E44814206F0FF06F5D1B245FE
S31508003F5071D0396ACB7ADB07CDD420460A7810F8B7
S31508003F600B3B01349B1A0131002BC4D114F8013BD9
S31508003F7011F8012B8442A3EB0203F5D1002BBAD129
S31508003F80184605B0BDE8F08FBB6A002BB6D06806A8
S31508003F9049D53A6994F80DA005F0BF057A62627BA7
S31508003FA0524542D1E17EA07E50EA012138D12078DF
S31508003FB0012100F03F00013800EB400A00EB8A0AB5
S31508003FC00395DFF8A0B02546CDF800801C4601927F
S31508003FD00846029713E0BAF1FE0F1DD8304601F0E5
S31508003FE00FF9804634F81A0001F00AF9804513D112
S31508003FF03046BA461A4B5B451FD01BF8011F6E1890
S315080040007678695C0AF1010741EA06260028E2D1BA
S315080040104FF6FF739E42EDD0DDF80080019A029FAD
S315080040209246FF266AE7AE42B9D0FF2666E7042025
S3150800403005B0BDE8F08F0020A3E723462C4621787B
S31508004040DDF800804906039D019A029F04D518B140
S3150800405033F81A30002BE3D1013DEEB292464DE714
S31508004060C4570008B85700082DE9F04FD0F820903B
S3150800407089B099F80B3013F0A00303D0062009B0D5
S31508004080BDE8F08FD0F82880B8F8006036B11E4633
S31508004090434633F8022F0136002AFAD1044623682C
S315080040A005A80C2249460193FFF714FA9DF81F301C
S315080040B0DD0772D5002389F80B300B22A36205A908
S315080040C048460125FFF706FA2B467E270DF1140E02
S315080040D0072203F00F0000F13001392988BF00F1EB
S315080040E037011B0902F1FF320EF8011DF1D108A9AB
S315080040F0114401F8147C002A00F0A98099F80010F0
S31508004100202908D0494603E011F8010F202802D0DB
S3150800411001339A42F8D109EB030108A8072A10448B
S3150800412098BF10F8140C03F101038CBF202001324C
S31508004130072B01F8010BF0D92046FFF7C7FE08BB8D
S315080041400135642D00F0F2800B2205A94846FFF7D9
S31508004150C1F9052D2B46B9D9A8F1020E3EF8022F52
S31508004160002AB3D0102102F0010000EB4303D80364
S3150800417044BF83F4883383F0210301394FEA52029E
S31508004180F1D1EBE704287FF47AAF9DF81F3089F860
S315080041900B309DF81F30C4F828809B0742D40021B5
S315080041A020464FF0010B2668FFF77CFC002848D113
S315080041B0054605E005462046FFF7C8FD002840D11C
S315080041C0A1693046FFF7B6F901210D44002838D118
S315080041D0E3691B78E52B01D0002BEBD1AB45EAD17F
S315080041E0BBF1010B35D1A1690198FFF7A3F90028A6
S315080041F07FF445AF0346E26902F1200102F8013B6C
S315080042008A42FBD10B22216AE069FFF763F9236A28
S31508004210E169DB7A012203F018030B73019B002086
S31508004220DA702CE7424B0C36A3FB063B00214FEA1B
S315080042309B0B20460BF1010B2668FFF733FC002881
S31508004240B6D0042808BF072009B0BDE8F08F13468A
S3150800425061E721692046A1EB4B11FFF723FC0028F3
S315080042607FF40DAF07463B46216A01F10B0011F8B2
S31508004270012BDD0145EA53031344814203F0FF0392
S31508004280F5D14FF6FF769A46A1690198FFF752F9DC
S31508004290074600287FF4F3AE5FFA8BF808F1FF3281
S315080042A0034602EB420002EB80024FF00F00E5697D
S315080042B02049D4F828C001F10C0EE87285F80DA043
S315080042C02F73AF76EF7601204FF0FF090EE03CF82A
S315080042D012302F182B54180A002B08BF33468E4568
S315080042E002F1010278700AD011F8010FB342EED13B
S315080042F02F188E4505F8009087F80190F4D1B3423F
S3150800430002D03CF812300BB948F04008019A012354
S3150800431085F800800021D3702046FFF717FD002896
S315080043207FF4ADAEBBF1010BAED15CE70720A6E684
S315080043304FECC44EB8570008012908D9F8B50568E6
S315080043400E466B690746994203D30220F8BD022040
S3150800435070475AB1012AF8D99342F6D91146284628
S315080043604FF0FF32FFF7F4FBB0B1F8BD284614E072
S31508004370314600222846FFF7EBFB0028F5D12B69CA
S315080043805A1C05D02A79013342F001022B612A71A1
S315080043906B699C4211D2264638683146FFF71EFBE8
S315080043A0044650B10128D0D0411C08D0012ECCD9E2
S315080043B06B699E42DCD30220F8BD0020F8BD0120BF
S315080043C0D3E700BF2DE9F04F0746D0F800A083B029
S315080043D00B780D462F2B01F10101F9D05C2BF7D094
S315080043E00021B96028781F2840F2308180B21F2842
S315080043F0BE6A2FD92F282DD05C282BD00121A9469B
S31508004400A6F10208012400F0D9FEF8B17F2809D8E0
S3150800441022281BD09C4A01E0984217D012F8013F87
S31508004420002BF9D128F8020F19F8010F631C1F2871
S3150800443012D92F2810D05C280ED0B3F5807F05D06E
S3150800444001211C4600F0BAFE0028DFD1062003B081
S31508004450BDE8F08F002401232B441A781D462F2A25
S3150800446003F10103F9D05C2AF7D01F288CBF4FF05F
S3150800447000094FF004094CB106EB440232F8023D3C
S31508004480202B01D02E2B04D1013CF7D100233380F9
S31508004490DCE7002326F814303B6A06EB440203F1F6
S315080044A00B00202103F8011B8342FBD1B31E4FF0FA
S315080044B0000801E008F1010833F8020F2028F9D0B6
S315080044C02E28F7D0B8F1000F01D049F0030913469A
S315080044D033F8022D2E2A01D0013CF9D100239B4640
S315080044E02B46354626465C46082208F1010870B375
S315080044F020281ED02E281AD0944221D2B0456DD03D
S315080045007F2875D82B2800F08480DFF884E101E045
S3150800451081427ED01EF8011F0029F9D1A0F1410180
S31508004520192900F29C804BF0020BC0B274E0B0452A
S3150800453004D049F0030935F81800D6E794424DD35C
S315080045400B2A70D0B0454BD049F0030948D91D460F
S315080045503B6A1978E5296ED0082A04BF4FEA8B0B07
S315080045605FFA8BFB0BF00C020C2A59D00BF00301F7
S31508004570032955D019F0020F0AD10BF0030BBBF132
S31508004580010F08BF49F01009042A08BF49F00809B5
S3150800459083F80B903846FFF799FC3B6ADB7A0028CC
S315080045A067D15A073FF553AFBB79DB064AD53B6956
S315080045B09AF80010C3F3080330335344D87E9A7E22
S315080045C0032942EA002202D0BA6028780EE7597D0C
S315080045D01B7D43EA012342EA0342F5E70B2A22D070
S315080045E04FEA8B0B5FFA8BFBB0460B220824A2E737
S315080045F000210192009300F0E1FD009B019AF0B1C1
S31508004600224949F00209084410F8800C00287FF472
S3150800461079AF49F003095F20396A085501348AE7FA
S3150800462049F00209A6E71D463B6A49F003091A78CC
S31508004630E52A97D10B22052119703B6A8CE749F0C8
S315080046400209E6E7052003B0BDE8F08F38463B6A65
S315080046508022DA7203B0BDE8F04FFFF723BAA0F163
S315080046606101192997BF2038C0B2C0B24BF0010BBF
S31508004670D2E704287FF4EBAE13F0040F08BF052039
S3150800468003B0BDE8F08F00BF24570008385700086C
S31508004690305700082DE9F843436A064601330D46AC
S315080046A01AD0836A18889C1C90B103F5007901F129
S315080046B01508002707E04C450AD008F8010F34F81A
S315080046C0020B013728B1002100F078FD0028F2D14D
S315080046D000272F440023BB7500210B46AC7D4FF005
S315080046E02E0CF0695A1CC35C202B1AD0052B08BF68
S315080046F0E523092A3CD0681843728CB9A3F141070F
S31508004700192F0CD8F769082A3F7B8CBF4FF0100E7B
S315080047104FF0080E17EA0E0F1CBF2033DBB2837565
S3150800472001310B2A1346DCD168182CB98475F36954
S315080047301B7B002B08BF284600234372F369DB7AEC
S315080047402B72F269D18B537F127F43EA012342EA27
S3150800475003232B60F269517E137E43EA0123AB8063
S31508004760F269D17D937D43EA0123EB80BDE8F883A6
S3150800477068180CB980F816C080F809C00131BAE784
S315080047802DE9F84FFF27044606683D46042006E053
S31508004790FF2500212046FFF7D9FA002857D1A1693D
S315080047A0002958D03046FEF7C5FE00284FD1E169EA
S315080047B00A78002A4AD0CB7AE52A03F03F03A37188
S315080047C0E6D02E2AE4D023F020000828E0D00F2BCC
S315080047D046D1500637D523694F7B02F0BF05636281
S315080047E091F80DE0BE45D3D1CA7E8B7E53EA0223EB
S315080047F026D10B782A4803F03F03013B012203EB3D
S31508004800430794464FF6FF7AD4F8289003EB8707B8
S3150800481000F10C0809E0FE2F12D89C4629F817303B
S31508004820013780452FD010F8012F8B1893F801B067
S315080048308B5C43EA0B23BCF1000FECD15345F0D057
S315080048407746FF25A5E7AA42A2D1C9E70420002397
S31508004850A361BDE8F88F0028F9D10020BDE8F88FDC
S315080048606DB901F10B0011F8013BEA0142EA550561
S315080048701D44814205F0FF05F5D1BD42EDD04FF04C
S31508004880FF336362E9E70B785B0604D5FE2FD7D8BA
S31508004890002329F81730013DEDB2774679E700BFC6
S315080048A0B857000810B584B004AB43F8041D01904E
S315080048B0184600911446FEF7C9FD031E11DB11497F
S315080048C051F823200AB100201070019A62B1002025
S315080048D01070019A41F823208AB1012C08D004B03F
S315080048E010BD0B2004B010BD104641F82320F6E792
S315080048F0024601A96846FEF7D7FE04B010BD104669
S31508004900EDE700BF70130020F0B593B0019148B3EE
S31508004910002302F01F06044615460360324603A923
S3150800492001A8FEF7C1FE08B113B0F0BD0399564AB7
S3150800493004AB079107A8019911920F93FFF742FD5F
S3150800494098B90F9B93F90B30002B54DB15F01C0F0D
S315080049501BD09DF8223013F0110F41D16F0710D5E7
S315080049600820E1E7092013B0F0BD15F01C0FDBD0D5
S315080049700428D9D107A8FFF777FB0028D4D146F039
S315080049800806350739D4039A0CE09DF82230D80674
S3150800499028D4A90701D5DA0722D42B07039A01D50B
S315080049A046F02006D16A0E9B216263621078DD7E8E
S315080049B0997E032841EA052116D0A160587FDD8B30
S315080049C0197F40EA052341EA03230020E3602674A1
S315080049D0226060746061E061D388A38013B0F0BD83
S315080049E00720A1E704209FE75D7D187D40EA0520A2
S315080049F041EA0041E1E7062096E70E9B0022612086
S31508004A004821187459749A73DA730E9B2025187600
S31508004A1059769A75DA750E9B0399DD720E9B0A789C
S31508004A20DD7E987E032A40EA052525D000229A765F
S31508004A30DA760878032804BF1A755A750E9B002281
S31508004A4001201A775A779A77DA77C8700DB9039AD8
S31508004A50A6E7039B07A82946DF6AFFF76DFC00282F
S31508004A607FF462AF39460398FEF764FD039A013D69
S31508004A70D560002894D057E7587D1A7D42EA00226F
S31508004A8045EA0245D2E700BF6C1100202DE9F04F38
S31508004A901E4683B000230F46336001A91446054617
S31508004AA0FEF7F8FC28B9687C18B92B7CD80703D41C
S31508004AB0072003B0BDE8F08F6B69EA68C3EB02080C
S31508004AC0A04528BFA046B8F1000F00F08780C3F3C1
S31508004AD0080105F1280900293DD10199B1F80AA074
S31508004AE00AF1FF3A1AEA532A41D0AB694A69023BEE
S31508004AF0023A934274D24A898C6A02FB0344002C18
S31508004B006ED05FEA582B54443BD00AEB0B03934212
S31508004B1088BFCAEB020B48785B4622463946FCF743
S31508004B20A7F800284AD12B7C5A0603D5E869001B4A
S31508004B3083454BD84FEA4B246B69B8EB04082344EA
S31508004B406B61336827442344336047D06B69C3F3EA
S31508004B5008010029C1D0C1F50074444528BF444660
S31508004B602831294422463846FEF7B4FCE4E743BB1D
S31508004B70A868012834D9411C20D003460199A861A8
S31508004B80B4E7EA69944214D02B7C5B060AD54878C8
S31508004B9001234946FCF7BEF880B92B7C019923F01E
S31508004BA040032B744878012322464946FCF760F8EF
S31508004BB020B96969EC61C1F30801CCE70120687482
S31508004BC077E7A9692868FEF709FFD2E707EB4020CF
S31508004BD04FF400724946FEF77DFCABE7002068E714
S31508004BE00220687465E700BF2DE9F04F1F4683B0C1
S31508004BF0002388463B6001A916460446FEF74AFC90
S31508004C0028B9607C18B9227C910703D4072003B021
S31508004C10BDE8F08F6369F34228BFDE43002E00F03B
S31508004C20898004F128094FE0019AB2F80AA00AF12E
S31508004C30FF3A1AEA532A0ED1002B74D1A06800282D
S31508004C407DD0012800F09980421C69D0A368A06134
S31508004C50019A03B9A060237C5B0654D4A369516901
S31508004C60023B02398B4280F088805089956A00FBA6
S31508004C700353002B00F081805FEA562B0AEB0305ED
S31508004C8036D00AEB0B03834288BFCAEB000B5B46A0
S31508004C90507841462A46FCF73DF8002840D1E1699C
S31508004CA0491B8B455DD84FEA4B256369E2682B445F
S31508004CB09A4238BF1A466361E2603B68761B2B440A
S31508004CC0A8443B6035D06369C3F308000028ABD01D
S31508004CD0C0F50075B54228BF3546283020442A4617
S31508004CE04146FEF7F7FB237C43F040032374DCE7D9
S31508004CF0E36960699D4202D0E368984227D3E5617B
S31508004D00C0F30800E4E750780123E2694946FCF756
S31508004D1001F828B9237C019A23F0400323749DE700
S31508004D200120607473E7A1692046FEF7A7FF0028F3
S31508004D3087D1227C42F020022274002067E7514680
S31508004D402046FEF79BFF00287FF47BAFF1E75078FB
S31508004D5001232A464946FBF78BFF0028E0D1606904
S31508004D60CDE708EB41214FF400724846FEF7B2FB47
S31508004D70237C23F04003237495E70220607446E7FA
S31508004D8070B50A2982B00E4605461AD06A68002A06
S31508004D9008DB541CAB183C2C1E7305DCAB686C6036
S31508004DA00133AB6002B070BD01AB224605F10C01C0
S31508004DB02868FFF719FF019B1C1B18BF4FF0FF342B
S31508004DC0ECE70D21FFF7DCFFE0E700BFF0B583B0A5
S31508004DD001A90446FEF75EFB002846D1227C02F0B4
S31508004DE0200303F0FF00002B3FD053060DD5019A90
S31508004DF00123507804F12801E269FBF78BFF0028AC
S31508004E0035D1237C23F040032374216A0198FEF7E9
S31508004E1091FB50BB636ADA7A42F02002DA72A26822
S31508004E202168C2F30720D8769A760978032920D014
S31508004E30E16801980D0A002219775D774FEA114E4D
S31508004E400F0E61260121482583F81EE0DF779A7543
S31508004E50DA759A74DA741E765D76C1700198FEF773
S31508004E6089FB237C23F02003237403B0F0BD0120C3
S31508004E70FBE7120C110A1A755975D9E710B582B0F5
S31508004E800446FFF7A3FF08B102B010BD01A92046EA
S31508004E90FEF700FB0028F7D1206002B010BD00BF66
S31508004EA070B582B00D4601A90446FEF7F3FA00284C
S31508004EB042D1607C00283FD1E368AB4204D2227C11
S31508004EC012F0020F08BF1D46002263696261002DB9
S31508004ED034D0019A568976023BB1013B6A1EB3FB70
S31508004EE0F6F1B2FBF6F28A425AD2A168002962D0DC
S31508004EF0A16131BB0D466669C6F30803002B64D071
S31508004F00E269954261D0237C5B063AD404F128060F
S31508004F10019B314658782A460123FBF7A9FE00284B
S31508004F2038D16669E368E5619E4268D9237CE66004
S31508004F3043F020032374002002B070BD284602B057
S31508004F4070BDB54214D843E02046FEF797FE0146E9
S31508004F5000283CD04A1C1DD001291ED9019B5B693B
S31508004F6099421AD26369AE423344A161636130D271
S31508004F70237CAD1B9807E7D42068FEF72FFD014672
S31508004F80E8E7019B04F12806587831460123FBF728
S31508004F90C1FE58B101206074CEE702206074CBE7E9
S31508004FA0724213406361ED1AA169A2E7237C23F0DC
S31508004FB040032374ACE72046FEF760FE012801464D
S31508004FC0EBD0431CE6D0A06092E7E368ACE7354631
S31508004FD06369EE18C5F30800666170B101988B1E07
S31508004FE04269023A9342D8D24289816A03FB021186
S31508004FF00029D2D001EB55257EE705467CE700203F
S315080050009AE700BF30B591B001900D46002205A978
S3150800501001A8FEF749FB044610B1204611B030BD81
S315080050200F4A02AB019905A80F920D93FFF7CAF92B
S3150800503004460028F1D10D9B93F90B30002B0ADBAF
S31508005040002DEAD00B9BA875002BE6D0294605A8AB
S31508005050FFF720FBE1E70624204611B030BD00BF6C
S315080050606C11002030B59DB00190022202A901A85A
S31508005070FEF71AFB029B069308B11DB030BD254A00
S3150800508003AB06A8019910920E93FFF79BF9002827
S31508005090F3D10E9B93F90B30002B05DB9DF81E20F0
S315080050A0D10703D50720E8E70620E6E7029D0D9914
S315080050B02878CC7E8B7E032843EA04241BD0D306AB
S315080050C009D406A8FEF7DAFE0028D6D1D4B9029884
S315080050D0FEF750FAD1E711A8002111951394FEF7AF
S315080050E0E1FC0028C9D111A8FFF74AFB0028D9D04E
S315080050F00428E6D0C1E7487D0B7D43EA002344EA4D
S315080051000344DCE70246214606A8FFF715F90028FE
S31508005110B3D1DCE76C1100202DE9F0418046174633
S31508005120054682B04E1E0024B4424FF0010212DA40
S3150800513001AB69463846FFF7A9FC019B6A1C012B9F
S3150800514009D19DF800300D2BEED00A2B2B7004F1F7
S3150800515001041546E8D1002C4FF0000314BF404661
S3150800516018462B7002B0BDE8F08100BF10B50446A2
S315080051700846217894B00023019002930393D1B195
S3150800518001A8FFF7FDFD14F8011F0029F8D1029ABE
S31508005190002A0CDB01986B4604A9FFF725FD30B9F8
S315080051A0029A009B9A4202D1039814B010BD4FF0A0
S315080051B0FF3014B010BD0A46EDE700BF7F2811D9AD
S315080051C089B910B40D4AC72303E0802914D032F8F0
S315080051D0023F98428CB201F10101F6D104F1800038
S315080051E080B210BC7047FF2804D8044B803833F8C7
S315080051F010007047002070470020F2E78458000826
S31508005200264AB0F5805F264B38BF134670B441F680
S315080052107D5138BF6121043381B188420ED333F8FA
S31508005220022C1E46D4B26518A8424FEA122207DBA2
S31508005230043372B133F8041C0029EED170BC7047F0
S31508005240082AFBD8DFE802F00E12181B1E212427B5
S315080052500A0006EB440336F81410DCE7A0F5E35021
S3150800526080B2EBE7411A33F81100E7E7411A01F07B
S315080052700103C01A80B2E1E7103880B2DEE72038B1
S3150800528080B2DBE7303880B2D8E71A3880B2D5E783
S31508005290083080B2D2E7503880B2CFE78459000888
S315080052A0C857000808B5074B044613B10021AFF3E9
S315080052B00080054B1868836A03B198472046FBF7B8
S315080052C09FFE00BF00000000785B00080E4B70B51B
S315080052D01E460E4C0025E41AA410A54204D056F822
S315080052E0253098470135F8E700F054F8084B094C83
S315080052F01E46E41AA4100025A54204D056F8253007
S3150800530098470135F8E770BDC0020020C0020020AA
S31508005310C0020020C4020020034B1B68186A034B16
S31508005320002808BF18467047500100205401002085
S3150800533008B5034B1868FFF7EFFFD0F8EC0008BD77
S315080053405001002082B001B901A93AB143B11378DE
S315080053500B601278101C18BF012003E0104601E00C
S315080053606FF0010002B0704703460244934202D030
S3150800537003F8011BFAE7704749B1FF2A85BF8A235C
S3150800538003600A704FF0FF3098BF01207047084647
S3150800539070470000F8B500BFF8BC08BC9E467047C9
S315080053A0F8B500BFF8BC08BC9E467047120110014C
S315080053B000000040501DAC6000010102030100001E
S315080053C0040309042603570069006E0055005300BC
S315080053D042002000420075006C006B00200044006B
S315080053E06500760069006300650000000902200078
S315080053F0010100C0320904000002FF00000407058D
S315080054008102400000070501024000001A034F0010
S31508005410700065006E0042004C00540020005500E4
S3150800542073006500720000002C03570069006E00C7
S315080054305500530042002000420075006C006B00C6
S31508005440200049006E007400650072006600610065
S31508005450630065006D61696E2E6300002F64656DDB
S315080054606F70726F675F6F6C696D6578696E6F5F75
S3150800547073746D33322E7372656300002F626F6F1B
S31508005480746C6F672E747874000000004F70656E38
S31508005490424C5400000008003F000000303A00006B
S315080054A02E2E2F2E2E2F2E2E2F536F757263652FAD
S315080054B066696C652E6300004669726D7761726570
S315080054C020757064617465207265717565737420E2
S315080054D064657465637465640A0D00004F70656ED3
S315080054E0696E67206669726D776172652066696C98
S315080054F06520666F722072656164696E672E2E2E4E
S31508005500000000004552524F520A0D004F4B0A0D3B
S31508005510000000005374617274696E6720746865D0
S315080055202070726F6772616D6D696E672073657141
S3150800553075656E63650A0D0050617273696E672042
S315080055406669726D776172652066696C6520746F2D
S315080055502064657465637420657261736520626C86
S315080055606F636B732E2E2E0045726173696E67200A
S31508005570000000002062797465732066726F6D20E2
S315080055806D656D6F727920617420307800000000B7
S3150800559052656164696E67206C696E652066726F14
S315080055A06D2066696C652E2E2E4552524F520A0D95
S315080055B000000000496E76616C6964206368656363
S315080055C06B73756D20666F756E642E2E2E4552525E
S315080055D04F520A0D0000000050726F6772616D6DC0
S315080055E0696E672000000000206279746573207474
S315080055F06F206D656D6F72792061742030780000B8
S3150800560057726974696E672070726F6772616D2070
S31508005610636865636B73756D2E2E2E00436C6F730E
S31508005620696E67206669726D776172652066696C56
S31508005630650A0D004669726D77617265207570643A
S31508005640617465207375636365737366756C6C79CD
S3150800565020636F6D706C657465640A0D0000000048
S315080056602E2E2F2E2E2F2E2E2F536F757263652FEB
S3150800567041524D434D335F53544D333246312F75A6
S3150800568073622E630000000000600008002000001E
S31508005690030000000080000800200000040000004D
S315080056A000A00008002000000500000000C0000857
S315080056B0002000000600000000E0000800200000AE
S315080056C00700000000000108002000000800000094
S315080056D00020010800200000090000000040010821
S315080056E0002000000A0000000060010800200000F9
S315080056F00B00000000800108002000000C000000DC
S3150800570000A00108002000000D00000000C00108EC
S31508005710002000000E00000000E001080020000044
S315080057200F000000222A3A3C3E3F7C7F0000000022
S315080057302B2C3B3D5B5D0000809A45418E418F8056
S315080057404545454949498E8F9092924F994F5555EF
S3150800575059999A9B9C9D9E9F41494F55A5A5A6A7D9
S31508005760A8A9AAABACADAEAFB0B1B2B3B4B5B6B733
S31508005770B8B9BABBBCBDBEBFC0C1C2C3C4C5C6C723
S31508005780C8C9CACBCCCDCECFD0D1D2D3D4D5D6D713
S31508005790D8D9DADBDCDDDEDFE0E1E2E3E4E5E6E703
S315080057A0E8E9EAEBECEDEEEFF0F1F2F3F4F5F6F7F3
S315080057B0F8F9FAFBFCFDFEFF01030507090E1012B6
S315080057C01416181C1E0000007D1D0100632C001E07
S315080057D09601A01E5A01001F0806101F0606201F64
S315080057E00806301F0806401F0606511F0700591FE6
S315080057F0521F5B1F541F5D1F561F5F1F601F080641
S31508005800701F0E00BA1FBB1FC81FC91FCA1FCB1F98
S31508005810DA1FDB1FF81FF91FEA1FEB1FFA1FFB1F12
S31508005820801F0806901F0806A01F0806B01F040060
S31508005830B81FB91FB21FBC1FCC1F0100C31FD01F42
S315080058400206E01F0206E51F0100EC1FF21F010019
S31508005850FC1F4E2101003221702110028421010013
S315080058608321D0241A05302C2F04602C0201672CC2
S315080058700601752C0201802C6401002D260841FFC3
S315080058801A030000C700FC00E900E200E400E0009B
S31508005890E500E700EA00EB00E800EF00EE00EC00A8
S315080058A0C400C500C900E600C600F400F600F20010
S315080058B0FB00F900FF00D600DC00A200A300A5004B
S315080058C0A7209201E100ED00F300FA00F100D100F3
S315080058D0AA00BA00BF001023AC00BD00BC00A1009E
S315080058E0AB00BB0091259225932502252425612529
S315080058F06225562555256325512557255D255C25A1
S315080059005B251025142534252C251C2500253C252A
S315080059105E255F255A255425692566256025502567
S315080059206C2567256825642565255925582552253A
S3150800593053256B256A2518250C25882584258C254D
S3150800594090258025B103DF009303C003A303C30397
S31508005950B500C403A6039803A903B4031E22C6030D
S31508005960B50329226122B10065226422202321235E
S31508005970F7004822B0001922B7001A227F20B20089
S31508005980A025A00061001A03E0001703F80007032A
S31508005990FF000100780100013001320106013901DA
S315080059A010014A012E017901060180014D004302CA
S315080059B081018201820184018401860187018701B0
S315080059C089018A018B018B018D018E018F0190015E
S315080059D09101910193019401F601960197019801AD
S315080059E098013D029B019C019D0120029F01A00197
S315080059F0A001A201A201A401A401A601A701A70171
S31508005A00A901AA01AB01AC01AC01AE01AF01AF011E
S31508005A10B101B201B301B301B501B501B701B801CE
S31508005A20B801BA01BB01BC01BC01BE01F701C00146
S31508005A30C101C201C301C401C501C401C701C8012E
S31508005A40C701CA01CB01CA01CD011001DD01010060
S31508005A508E01DE011201F3010300F101F401F401E4
S31508005A60F8012801220212013A020900652C3B02BC
S31508005A703B023D02662C3F024002410241024602B9
S31508005A800A015302400081018601550289018A01F3
S31508005A9058028F015A0290015C025D025E025F02A3
S31508005AA0930161026202940164026502660267025A
S31508005AB0970196016A02622C6C026D026E029C01C5
S31508005AC0700271029D01730274029F0176027702C9
S31508005AD0780279027A027B027C02642C7E027F02BB
S31508005AE0A60181028202A901840285028602870232
S31508005AF0AE014402B101B20145028D028E028F0247
S31508005B0090029102B7017B030300FD03FE03FF0326
S31508005B10AC0304008603880389038A03B1031103CF
S31508005B20C2030200A303A303C4030803CC030300B0
S31508005B308C038E038F03D8031801F2030A00F903B6
S31508005B40F303F403F503F603F703F703F903FA037C
S31508005B50FA033004200350041007600422018A0463
S31508005B603601C1040E01CF040100C004D00444016B
S31508005B706105260400000000F00000204300504F95
S31508005B80534958002E0000202020202020202020C5
S31508005B9028282828282020202020202020202020CF
S31508005BA020202020202020881010101010101010FF
S31508005BB01010101010101004040404040404040443
S31508005BC004101010101010104141414141410101CB
S31508005BD001010101010101010101010101010101A7
S31508005BE001011010101010104242424242420202B5
S31508005BF00202020202020202020202020202020277
S31508005C000202101010102000000000000000000022
S31508005C100000000000000000000000000000000076
S31508005C200000000000000000000000000000000066
S31508005C300000000000000000000000000000000056
S31508005C400000000000000000000000000000000046
S31508005C500000000000000000000000000000000036
S31508005C600000000000000000000000000000000026
S31508005C700000000000000000000000000000000016
S31108005C800000000000000000000000000A
S30D08005C8CBCA4FF7F0100000023
S31508005C941C0353004500520031003200330034001F
S31508005CA4350036003700380039003000EC53000858
S31508005CB4200000000D030008310300082104000831
S31508005CC4B5020008B9020008F9020008FD02000836
S31508005CD4DD030008E9030008F503000800000000D6
S31508005CE440000000051E000891020008051E000871
S31508005CF4051E0008051E0008051E0008051E0008E6
S31508005D04051E0008A9020008FE5300080900000041
S31508005D14AC53000812000000C05300080400000039
S31508005D240C5400081A000000C4530008260000009A
S31508005D34000000201C000000285400082C00000065
S31508005D440301000075020008051E0008051E000868
S31508005D54051E0008051E0008051E0008051E000885
S31508005D6479020008051E0008051E0008051E00081D
S31508005D74051E0008051E0008051E0008010400008B
S31508005D840000000000000000000000000000000001
S31508005D9400000000000000000000000000000000F1
S31508005DA400000000000000000000000000000000E1
S31508005DB400000000000000000000000000000000D1
S31508005DC400000000000000000000000000000000C1
S31508005DD400000000000000000000000000000000B1
S31508005DE4F00000204300000000000000000000004E
S31508005DF40000000000000000000000000000000091
S31508005E04000000004300000000000000000000003D
S31508005E140000000000000000000000000000000070
S31508005E24000000004300000000000000000000001D
S31508005E340000000000000000000000000000000050
S31508005E4400000000430000000000000000000000FD
S31508005E540000000000000000000000000000000030
S31508005E6400000000430000000000000000000000DD
S31508005E740000000000000000000000000000000010
S31508005E8400000000430000000000000000000000BD
S31508005E9400000000000000000000000000000000F0
S31508005EA4000000004300000000000000000000009D
S31508005EB400000000000000000000000000000000D0
S31508005EC4000000007953000845530008000000004C
S31508005ED4865B0008845B0008855B0008855B000810
S31508005EE4855B0008855B0008855B0008855B000800
S31508005EF4855B0008855B0008855B0008FFFFFFFFDC
S31508005F04FFFFFFFFFFFFFFFFFFFF000001004153F4
S31508005F14434949000000000000000000000000009A
S31508005F2400000000000000000000000000004153CB
S31508005F34434949000000000000000000000000007A
S31508005F44000000000000000000000000000000003F
S30D08005F5411010008ED00000828
S70508000000F2
